:020000040800F2
:10000000E0120020C10100080F390008B9350008CE
:100010000D390008A7060008B943000800000000D9
:10002000000000000000000000000000133900087C
:100030007D0700080000000011390008153900088C
:10004000DB010008DB010008DB010008DB01000820
:10005000DB010008DB010008DB010008DB01000810
:10006000DB010008DB010008DB010008DB01000800
:10007000DB010008A9060008DB010008DB0100081D
:10008000DB010008DB010008DB010008DB010008E0
:10009000DB010008DB010008DB010008DB010008D0
:1000A000DB010008DB010008DB010008DB010008C0
:1000B000DB010008D9390008DB010008DB0100087A
:1000C000DB010008DB010008DB010008DB010008A0
:1000D000DB010008AD430008DB010008DB0100087C
:1000E000DB010008DB010008DB010008DB01000880
:1000F000DB010008DB010008DB010008DB01000870
:10010000DB010008DB010008DB010008DB0100085F
:10011000DB010008DB010008DB010008DB0100084F
:10012000DB010008B5060008C1060008DB01000875
:10013000DB010008DB010008DB010008DB0100082F
:10014000DB010008DB010008DB010008DB0100081F
:10015000DB010008DB010008CD060008DB01000818
:10016000DB010008DB010008DB010008DB010008FF
:10017000DB010008DB010008DB01000800000000D3
:10018000DB010008DB010008DB010008DB010008DF
:10019000DB010008DB010008DB010008DB010008CF
:1001A000DB010008DB010008DB010008DFF80CD0F0
:1001B00000F006FA0048004799450008E0120020C8
:1001C0000648804706480047FEE7FEE7FEE7FEE7F1
:1001D000FEE7FEE7FEE7FEE7FEE7FEE7BD390008C3
:1001E000AD0100082DE9F05F0546002092469B46D0
:1001F00088460646814640241BE02846414647463D
:10020000224600F000F953465A46C01A914110D3D5
:1002100011461846224600F0E7F82D1A67EB010850
:100220004F4622460120002100F0DEF817EB0009BE
:100230004E41201EA4F10104DFDC484631462A4627
:100240004346BDE8F09FD2B201E000F8012B491E01
:10025000FBD270470022F6E710B513460A46044663
:100260001946FFF7F0FF204610BD70B5064604F0B2
:10027000C5F8046805460A220021304600F0D3F88C
:100280002C6070BD2DE9F04D81EA030404F0004BB1
:1002900021F0004514464FF0000A23F0004150EAD7
:1002A000050220D054EA01021DD0C5F30A570246C8
:1002B000C5F31303C1F31300C1F30A5640F48015CC
:1002C00043F48013A7EB0608101BD64608F2FD384E
:1002D00073EB050002D308F1010801E092185B41BD
:1002E000B8F1000F03DA00200146BDE8F08D0020D0
:1002F0004FF48011064684460EE0171B73EB05078A
:1003000005D3121B63EB050306434CEA010C4908B5
:100310004FEA300092185B4150EA0107EDD152EAF2
:10032000030012D082EA040083EA0501084305D0E5
:10033000101BAB4106D20122002306E000224FF041
:10034000004302E06FF0010253101AEB06004CEB81
:10035000085110EB0A0041EB0B01BDE8F04D00F035
:10036000D1B80EB5C10F80EAE0700844CA07002179
:1003700040F233438DE80E000A460B4600F0D1F8F8
:1003800003B000BD01F0004330B421F0004150EA59
:10039000010206D00A0DA2F56072C1F31301002A12
:1003A00002DC30BC00207047440F44EAC104C100A5
:1003B000E01830BC00EBC25000F06DB830B50B4611
:1003C000014600202022012409E021FA02F59D4285
:1003D00005D303FA02F5491B04FA02F52844151E59
:1003E000A2F10102F1DC30BD202A04DB203A00FA40
:1003F00002F1002070479140C2F1200320FA03F37C
:10040000194390407047202A04DB203A21FA02F079
:100410000021704721FA02F3D040C2F1200291403E
:100420000843194670472DE9F04791460F4680462C
:100430000446002614F8015B2DB100F0D3F80068E3
:10044000405DC007F6D12B2D02D02D2D18D0641E93
:100450004A463946204600F0C9F827B13968A1421A
:1004600001D1C7F8008071054FF002040BD540425E
:10047000002803DD03F0C2FF0460A007BDE8F08799
:1004800046F48066E4E70028F8DA03F0B7FF04607A
:100490006FF00040F2E70029A8BF7047401C4900F8
:1004A00008BF20F00100704710B4B0FA80FC00FAD9
:1004B0000CF050EA010404BF10BC704749B1CCF104
:1004C000200421FA04F411FA0CF118BF0121214390
:1004D0000843A3EB0C01CB1D4FEA00614FEA10204B
:1004E00042BF002010BC704700EBC35010440029ED
:1004F000A4BF10BC7047401C490008BF20F0010099
:1005000010BC704710B5141E73F1000408DA401CCB
:1005100041F1000192185B411A4301D120F0010022
:1005200010BD2DE9F04D92469B4611B1B1FA81F212
:1005300002E0B0FA80F220329046FFF755FF044601
:100540000F4640EA0A0041EA0B0153465A46084367
:1005500013D0114653EA010019D0C8F140025046A9
:10056000FFF751FF05460E46504659464246FFF7F3
:100570003BFF084305D0012004E020463946BDE892
:10058000F08D0020054346EAE0762C4337430A9875
:100590006305E40AA0EB08000022FD0A44EA475480
:1005A0000A3002D500200146E9E70105101969412A
:1005B000DDE9084500196941BDE8F04DA2E70000FA
:1005C000064C074D06E0E06840F0010394E80700A0
:1005D00098471034AC42F6D3FFF7ECFDFC48000816
:1005E0001C49000800487047F84800082DE9F05FF2
:1005F00082460078002715468B460AF10104B94669
:10060000302801D09DB113E014F8010B01277828A0
:1006100003D0582801D045B10AE00DB1102D07D103
:100620000027102514F8010B02E0082500E00A2538
:100630000026B0460EE005FB080005FB06F1012789
:1006400001EB10461FFA80F8B6F5803F00D3B9469B
:1006500014F8010B294600F018F80028EBDABBF17A
:10066000000F05D00FB1641E00E05446CBF80040E7
:10067000B9F1000F06D003F0C1FE02210160C81ECF
:10068000BDE8F09F48EA0640FAE73A2800D2303841
:1006900020F02002412A01D3A2F13700884201D381
:1006A0004FF0FF307047FEE7014800F07BB80000D4
:1006B000DC000020014800F075B800009C0100201B
:1006C000014800F06FB80000FC010020014800F074
:1006D00069B800003C0100200168CAB2103A182332
:1006E000B2FBF3F2064B9B5CC3656FF30901032A6F
:1006F00002D9091D816500E08165806D70470000A9
:100700005448000810B5014600208A6A8B694FF0F2
:10071000C074002B0ED0B3F5005F1AD062B3012A6B
:100720002AD0022A28D0032A03D1C96AC90100D5D8
:10073000012010BD1AB1012A06D0022AF9D1C96AD6
:10074000C901F6D5012010BDC96AA142FBD1012023
:1007500010BD52B1012A0AD0022A06D0032AF7D1CD
:10076000C96AA142F4D1012010BD012010BDC96A9F
:10077000C901FBD5012010BD012010BD7047704795
:1007800090F83510022903D080214165012070477F
:10079000052180F835100068016821F00101016031
:1007A000002070472DE9F84304464FF00009CDF8CA
:1007B00000906F484FF416510068B0FBF1F7A56D3B
:1007C0002E6894F85C00082202FA00F1314210D041
:1007D0002068016849070CD5016821F00401016017
:1007E00094F85C0002FA00F1A960606D40F001002D
:1007F000606594F85C104FF0010808FA01F030428F
:1008000008D021684969090604D5A860606D40F0E8
:100810000200606594F85C1004208840304208D0E3
:1008200021680968890704D5A860606D40F004005C
:10083000606594F85C1010208840304220D0216818
:10084000096809071CD5A8602068016849030CD510
:100850000068000304D4216C91B1204688470FE062
:10086000A16C69B1204688470AE00168C90503D434
:10087000016821F008010160216C09B12046884718
:1008800094F85C102020884030424CD021680968E0
:10089000C90648D5A86094F8350005280BD0206813
:1008A0000168490330D50068000328D4616C51B356
:1008B0002046884737E02068016821F01601016072
:1008C0002068416921F080014161206C08B9A06C69
:1008D00020B12068016821F00801016094F85C10E3
:1008E0003F208840A86084F8349084F83580216DDA
:1008F00000293BD001B02046BDE8F0430847E16B3A
:1009000009B1204688470EE00168C90507D401688F
:1009100021F01001016084F8349084F83580E16B97
:1009200009B120468847606D00281FD0606DC00760
:1009300014D0052084F835002068016821F00101F9
:1009400001600098401C0090B84203D820680068FD
:10095000C007F6D184F8349084F83580E16C002922
:1009600004D001B02046BDE8F0430847BDE8F88355
:100970001C0000202DE9F041044600F073FB054601
:10098000002C7CD0A149206888423ED09F49183174
:1009900088423AD09D493031884236D09B4948310F
:1009A000884232D09949603188422ED097497831B7
:1009B00088422AD095499031884226D09349A8315F
:1009C000884222D0924988421FD0914918318842EA
:1009D0001BD08F493031884217D08D494831884229
:1009E00013D08B49603188420FD0894978318842D1
:1009F0000BD087499031884207D08549A831884279
:100A000003D0B82183A003F0B7FD6068C0B1B0F196
:100A1000007F15D0B0F1806F12D0B0F1C06F0FD051
:100A2000B0F1006F0CD0B0F1206F09D0B0F1406F81
:100A300006D0B0F1606F03D0B92176A003F09CFD21
:100A4000A06838B1402805D0802803D0BA2171A011
:100A500003F092FDE068B0F5007F04D018B1BB212F
:100A60006CA003F089FD2069B0F5806F04D018B147
:100A7000BC2168A003F080FD606958B100E070E01F
:100A8000B0F5006F06D0B0F5805F03D0BD2161A046
:100A900003F072FDA06948B1B0F5005F06D0B0F573
:100AA000804F03D0BE215BA003F066FDE06940B13A
:100AB000B0F5807F05D0202803D0BF2155A003F0DA
:100AC0005BFD206A60B1B0F5803F09D0B0F5003F12
:100AD00006D0B0F5403F03D0C0214EA003F04CFD3E
:100AE000606A28B1042803D0C1214AA003F044FD64
:100AF000606A002829D0A06A48B1012807D00228DE
:100B000005D0032803D0C62142A003F035FDE06ADA
:100B100060B1B0F5000F09D0B0F1807F06D0B0F120
:100B2000C07F03D0C7213BA003F026FD206B60B13E
:100B3000B0F5001F09D0B0F5800F06D0B0F5C00F9A
:100B400003D0C82133A003F017FD002684F83460D9
:100B5000022084F835002068016821F0010101605D
:100B60000DE00120BDE8F08100F07CFA401B052873
:100B700005D920206065032084F83500F2E720685D
:100B80000068C007F0D121680A6830480240D4E903
:100B900001031843D4E903352B4318436369184311
:100BA000A3691843E3691843236A18431043626A30
:100BB000042A03D1D4E90B231A43104308602068A8
:100BC000406920F00701656A28460D430127042883
:100BD0000DD1A06A0543E06A48B12046FFF792FDB7
:100BE00028B14020606584F835700120BAE720689C
:100BF00045612046FFF770FD94F85C203F2191404D
:100C00008160666584F835700020ABE710600240B3
:100C1000106402402E2E2F447269766572732F5332
:100C2000544D3332463478785F48414C5F447269A2
:100C30007665722F5372632F73746D333266347816
:100C4000785F68616C5F646D612E63003F8010F0B7
:100C50002DE9F84F04460D46AA48844221D0AA48FF
:100C600084421ED0A94884421BD0A948844218D08F
:100C7000A848844215D0A848844212D0A74884428C
:100C80000FD0A74884420CD0A648844209D0A64879
:100C9000844206D0A548844203D0B321A4A003F027
:100CA0006BFC28680104090C01D0000C03D0B421AE
:100CB0009FA003F061FC6868F8B101281DD01128DD
:100CC0001BD0022819D0122817D0A849884214D066
:100CD000A749884211D0A74988420ED0A649884228
:100CE0000BD0A649884208D0A549884205D00328E0
:100CF00003D0B5218EA003F03FFCA86838B10128CD
:100D000005D0022803D0B62189A003F035FC0026C7
:100D10004FF0030A4FF00F0B4FF0010808FA06F8E6
:100D20002F6807EA080747457ED16868012805D083
:100D3000022803D0112801D012281DD1E86848B13B
:100D4000012807D0022805D0032803D0C82178A0A5
:100D500003F012FCA16870000AFA00F29143EA68FD
:100D600082400A43A260606820EA08002979C1F342
:100D70000011B14001436160E0684FEA46090AFA98
:100D800009F820EA0800A96801FA09F10143E160C5
:100D90006868022801D0122830D1286908B30928D0
:100DA0001FD001281DD002281BD0032819D00428E9
:100DB00017D0052815D0062813D0072811D00828E9
:100DC0000FD00A280DD00B280BD00C2809D00D28E5
:100DD00007D00F2805D00E2803D0E02154A003F03F
:100DE000CBFBF00804EB8000026A7107C90E0BFA16
:100DF00001F39A432B698B4013430362206820EA76
:100E00000800297901F0030101FA09F10143216089
:100E10006868C0006FD55B48016841F4804101609B
:100E2000006800F4804000E065E00090564826F03D
:100E300003010A18D2F80838B007010F0BFA01F0C5
:100E400083433048844201D100202DE02E48844263
:100E500001D1012028E02D48844201D1022023E065
:100E60002B48844201D103201EE02A48844201D14C
:100E7000042019E02848844201D1052014E02748C5
:100E8000844201D106200FE02548844201D1072089
:100E90000AE02448844201D1082005E02248844227
:100EA00001D1092000E00A2088401843C2F8080850
:100EB00036490868B8436A68D20300D538430860E9
:100EC0003249091D0868B8436A68920300D538435F
:100ED00008602E4908310868B8436A68D20200D514
:100EE0003843086029490C310868B8436A6892029F
:100EF00000D538430860761C102EFFF40DAFBDE816
:100F0000F88F000000000240000402400008024088
:100F1000000C024000100240001402400018024081
:100F2000001C024000200240002402400028024031
:100F30002E2E2F447269766572732F53544D3332BF
:100F4000463478785F48414C5F4472697665722F09
:100F50005372632F73746D3332663478785F6861CF
:100F60006C5F6770696F2E63000000000000111055
:100F700000002110000031100000121000002210AB
:100F8000000032104438024000300140003C014073
:100F900070B505460C46002C04D14FF4DB7106A059
:100FA00003F0EAFA686934EA000001D0AC6170BD70
:100FB0002004A86170BD00002E2E2F447269766552
:100FC00072732F53544D3332463478785F48414C16
:100FD0005F4472697665722F5372632F73746D3339
:100FE00032663478785F68616C5F6770696F2E6312
:100FF0000000000070B506460C461546002C04D1D2
:1010000040F29F1108A003F0B7FA35B1012D04D0CA
:101010004FF4D07104A003F0AFFA0DB1B46170BD0C
:101020002004B06170BD00002E2E2F4472697665D9
:1010300072732F53544D3332463478785F48414CA5
:101040005F4472697665722F5372632F73746D33C8
:1010500032663478785F68616C5F6770696F2E63A1
:101060000000000001488068704700001000002068
:1010700002488168027811448160704710000020A6
:1010800010B50B48016841F400710160016841F43A
:1010900080610160016841F480710160032000F00B
:1010A000C7F8002000F006F800F026F8002010BD78
:1010B000003C024070B504460D4D4FF47A7128781B
:1010C000B1FBF0F00B490968B1FBF0F000F03CFD1A
:1010D00008B1012070BD102C07D200222146501EFD
:1010E00000F056F86C60002070BD012070BD00005B
:1010F000100000201C00002008B50A48016841F4D7
:1011000080410160006800F4804000900548001FA5
:10111000016841F080510160006800F0805000904B
:1011200008BD00004438024010B50446002C03DA24
:10113000BE2108A003F020FA002C09DB04F01F01F7
:10114000012088406109890001F1E021C1F8000116
:1011500010BD00002E2E2F447269766572732F53D6
:10116000544D3332463478785F48414C5F4472695D
:101170007665722F5372632F73746D3332663478D1
:10118000785F68616C5F636F727465782E630000CE
:101190002DE9F04107460D461646102E03D3AA212D
:1011A00013A003F0E9F9102D03D3AB2110A003F035
:1011B000E3F91E480068C0F30223C3F10704042CBE
:1011C00000D90424181D072801D2002300E0DB1EEB
:1011D000012000FA04F1491E294099409840401E20
:1011E000304001433846BDE8F04103F0F7B8000055
:1011F0002E2E2F447269766572732F53544D3332FD
:10120000463478785F48414C5F4472697665722F46
:101210005372632F73746D3332663478785F68610C
:101220006C5F636F727465782E6300000CED00E0F4
:1012300010B50446072C0BD0062C09D0052C07D07E
:10124000042C05D0032C03D0922108A003F094F9BC
:1012500004F00701144A10684FF6FF03184040EAF3
:10126000012012490843106010BD00002E2E2F44AB
:101270007269766572732F53544D333246347878E1
:101280005F48414C5F4472697665722F5372632FD9
:1012900073746D3332663478785F68616C5F636F46
:1012A000727465782E6300000CED00E00000FA0512
:1012B0002DE9F8431848016841F080510160006849
:1012C00000F080500090DFF854800127C8F840708B
:1012D000FFF7C8FE05464FF47A76114C07E0FFF79A
:1012E000C1FE401BB04202D90320BDE8F88360680C
:1012F000C003F4D5C8F84470FFF7B4FE054606E015
:10130000FFF7B0FE401BB04201D90320EDE7606853
:101310008003F5D50020E8E74038024000000E4287
:10132000007000402DE9F04705460C46002D40D0E6
:101330002868401E0E2804D940F2512182A003F0F3
:101340001BF914B3012C20D0022C1ED0032C1CD06E
:10135000042C1AD0052C18D0062C16D0072C14D02B
:10136000082C12D0092C10D00A2C0ED00B2C0CD02B
:101370000C2C0AD00D2C08D00E2C06D00F2C04D02B
:1013800040F2522170A003F0F7F8DFF8F481D8F8AA
:101390000000E7B200F00F00A0420CD288F8007005
:1013A000D8F8000000F00F00A04204D00120BDE8F2
:1013B000F0870120FBE72868724E810729D5400796
:1013C00003D5306840F4E05030602878000703D53A
:1013D000306840F460403060A868A0B1802812D026
:1013E000902810D0A0280ED0B0280CD0C0280AD049
:1013F000D02808D0E02806D0F02804D040F275218B
:1014000051A003F0B9F83068A96820F0F000084353
:1014100030602878C0073ED0686850B1012808D0F5
:10142000022806D0032804D04FF41F7146A003F011
:10143000A3F8544968680839012808D002280BD05D
:10144000032809D0096889070BD40120AFE7096890
:10145000890306D40120AAE70968890101D4012083
:10146000A5E7316821F0030101433160FFF7FAFD80
:10147000814641F2883A07E0FFF7F4FDA0EB09004E
:10148000504501D9032092E73068696800F00C00EC
:10149000B0EB810FF0D1D8F8000000F00F00A042AF
:1014A00009D988F80070D8F8000000F00F00A042B9
:1014B00001D001207BE728784FF4805440074FF497
:1014C000A0574FF4C0584FF4E05914D5E86860B104
:1014D000A0420AD0B84208D0404506D0484504D0C2
:1014E00040F2BA2118A003F047F83068E96820F408
:1014F000E050084330602878000715D5286960B1AE
:10150000A0420AD0B84208D0404506D0484504D091
:1015100040F2C1210CA003F02FF83068296920F4B3
:10152000604040EAC100306000F05AF83168164A65
:10153000C1F30311515CC8401449086014480068A5
:10154000FFF7B8FD002032E72E2E2F447269766532
:1015500072732F53544D3332463478785F48414C80
:101560005F4472697665722F5372632F73746D33A3
:1015700032663478785F68616C5F7263632E6300F3
:10158000003C0240083802405C4800081C00002073
:101590001400002001480068704700001C00002073
:1015A00000B5FFF7F7FF04490968044AC1F3822137
:1015B000515CC84000BD0000083802406C4800087B
:1015C00000B5FFF7E7FF04490968044AC1F3423157
:1015D000515CC84000BD0000083802406C4800085B
:1015E00010B51748006810F00C01164816D0164BBD
:1015F000042912D0082911D1114C241F216801F0AF
:101600003F02216849020AD52068C0F38810A0FB78
:1016100003010023FEF7E6FD09E0184610BD21682E
:101620000023C1F38811A1FB0001FEF7DBFD216857
:10163000C1F30141491C4900B0FBF1F010BD0000AD
:10164000083802400024F40040787D012DE9F84F6D
:101650000446002C27D020680F2803D9E821F3A0E6
:1016600002F08AFF2078FF4FC007A7F1040561D080
:1016700060684FF480364FF4A02838B1B04205D0EE
:10168000404503D0ED21E9A002F076FFF548001DAA
:101690000168C1F3810101290BD00068C0F381000A
:1016A000022803D00CE00120BDE8F88F3868400222
:1016B00006D5286880033DD5606860BB0120F3E74C
:1016C0006068B04204D1286840F48030286012E09D
:1016D000404508D1286840F480202860286840F4FC
:1016E0008030286007E0286820F48030286028686F
:1016F00020F480202860606870B1FFF7B3FC0646D4
:1017000006E0FFF7AFFC801B642801D90320CBE77C
:1017100028688003F5D50DE0FFF7A4FC064606E037
:10172000FFF7A0FC801B642801D90320BCE72868D0
:101730008003F5D42078CC4E80074FF000095AD5AD
:10174000E06830B1012804D040F21F11B7A002F0C8
:1017500013FF20691F2804D94FF49071B3A002F041
:101760000BFFC048001D016811F00C0F07D0006886
:10177000C0F38100022812D1386840020FD42868D3
:10178000800704D5E068012801D001208CE7286893
:10179000216920F0F80040EAC10028602BE0E068F1
:1017A000C0B101203060FFF75DFC804607E0FFF725
:1017B00059FCA0EB0800022801D9032074E728682F
:1017C0008007F4D52868216920F0F80040EAC100BC
:1017D000286010E0C6F80090FFF744FC804607E060
:1017E000FFF740FCA0EB0800022801D903205BE7CB
:1017F00028688007F4D42078000734D5606930B1B8
:10180000012804D04FF4B07188A002F0B5FEDFF8D3
:1018100054A2964960690AF1700A90B101200860EB
:10182000FFF720FC804607E0FFF71CFCA0EB080058
:10183000022801D9032037E7DAF800008007F3D542
:1018400011E0C1F80090FFF70DFC804607E0FFF7BC
:1018500009FCA0EB0800022801D9032024E7DAF8EC
:1018600000008007F3D42078400772D54FF00008BD
:10187000A06840B1012806D0052804D04FF4C671F5
:101880006AA002F079FE77483C300068C0000BD4B3
:1018900074483C30016841F080510160006800F0FC
:1018A000805000904FF00108DFF8C4B1DBF8000071
:1018B000C00515D4DBF8000040F48070CBF80000C0
:1018C000FFF7D0FB824607E0FFF7CCFBA0EB0A0056
:1018D000022801D90320E7E6DBF80000C005F3D5B4
:1018E000DFF880B1A0680BF16C0B012813D005283C
:1018F00018D0DBF8000020F00100CBF80000DBF886
:10190000000020F00400CBF80000A06838B3FFF717
:10191000A9FB82461EE0DBF8000040F00100CBF896
:101920000000F2E7DBF8000040F00400CBF8000014
:10193000DBF8000040F00100CBF80000E5E7FFF71E
:1019400091FBA0EB0A0141F28830814202D90320C9
:10195000AAE61FE0DBF800008007F0D511E0FFF7F2
:1019600081FB824609E0FFF77DFBA0EB0A0141F213
:101970008830814201D9032096E6DBF80000800719
:10198000F1D4B8F1010F05D136483C30016821F09F
:1019900080510160A06940B1012806D0022804D01E
:1019A00040F2CF1121A002F0E7FDA069002875D018
:1019B0002C49091D0968C1F3810102296FD0022851
:1019C00005D0C6F86090FFF74DFB044695E0E0694E
:1019D00038B1B0F5800F04D04FF4EC7113A002F0D1
:1019E000CBFD206A3F2804D940F2D9110FA002F0A4
:1019F000C3FD606A3238B0F5BF7F04D94FF4ED7192
:101A00000AA002F0B9FDA06A02280AD0042808D072
:101A1000062806D0082804D040F2DB1103A002F00B
:101A2000ABFDE06A801E0D282AD923E02E2E2F441C
:101A30007269766572732F53544D33324634787819
:101A40005F48414C5F4472697665722F5372632F11
:101A500073746D3332663478785F68616C5F72637B
:101A6000632E63000438024000004742800E474264
:101A7000007000404FF4EE71AFF2500002F07CFDB8
:101A8000C6F86090FFF7EEFA804609E0FFF7EAFA41
:101A9000A0EB0800022803D9032005E652E030E05D
:101AA00028688001F2D4D4E907010843616AA26A78
:101AB0004FF0FF33890103EB520241EA0241084330
:101AC00094F82C1040EA0160386001203066FFF77E
:101AD000C9FA044606E0FFF7C5FA001B022801D93F
:101AE0000320E1E528688001F5D52BE0FFF7BAFA7D
:101AF000001B022801D90320D6E528688001F5D40F
:101B000020E001281CD03868E26900F4800191428D
:101B100014D1226A00F03F0191420FD147F6C07103
:101B2000626A0140914209D1A26A00F440319142B7
:101B300004D1E16A00F07060884203D00120B3E56F
:101B40000120B1E50020AFE510B5401EB0F1807F67
:101B500001D3012010BD4FF0E02460610F21601718
:101B600002F03CFC0020A06107202061002010BD95
:101B70007047704770B505460C463F492868884253
:101B800007D03E49884204D040F2A1613CA002F057
:101B9000F3FC2068B0F5006F05D020B140F2A261DF
:101BA00037A002F0E9FC6068B0F5806F05D020B185
:101BB00040F2A36132A002F0DFFCA06868B1B0F58A
:101BC000807F0AD0B0F5007F07D0B0F5407F04D009
:101BD00040F2A4612AA002F0CFFCE068FF2804D9FB
:101BE00040F2A56126A002F0C7FC2069B0F5805F35
:101BF00005D020B140F2A66121A002F0BDFC6069D1
:101C000038B1B0F5005F04D040F2A7611CA002F02B
:101C1000B3FCE069B0F5804F05D020B14FF4D56139
:101C200017A002F0A9FC95F83C00012822D0012061
:101C300085F83C00E0680021A26820F44070104361
:101C4000626820F480601043226820F40060104332
:101C5000226920F480501043626920F40050104340
:101C6000E26920F4804010432A68506485F83C10F3
:101C7000002070BD022070BD000001400004014042
:101C80002E2E2F447269766572732F53544D333262
:101C9000463478785F48414C5F4472697665722FAC
:101CA0005372632F73746D3332663478785F686172
:101CB0006C5F74696D5F65782E6300002DE9F05FDD
:101CC00004460D46394E2068394FDFF8E880DFF8CA
:101CD000E890DFF8E8A04FF0804BB04215D05845AF
:101CE00013D0B84211D040450FD048450DD04FEA2F
:101CF000B641884209D03249884206D0504504D0C6
:101D000040F264612FA002F037FC286890B11028DF
:101D100010D020280ED030280CD040280AD05028CF
:101D200008D0602806D0702804D040F2656125A054
:101D300002F022FC6868802805D020B140F266617C
:101D400020A002F019FC94F83C0001282CD00122BC
:101D500084F83C20022084F83D00206843688168B4
:101D600023F0700C2B6843EA0C0343602068B042F8
:101D70000FD058450DD0B8420BD0404509D048454A
:101D800007D0504505D01E4B984202D01D4B9842BB
:101D900004D121F080036968194381603C3462708A
:101DA00000202070BDE8F09F0220FBE7000001400A
:101DB0000004004000080040000C00400004014006
:101DC000001400402E2E2F447269766572732F53D3
:101DD000544D3332463478785F48414C5F447269E1
:101DE0007665722F5372632F73746D333266347855
:101DF000785F68616C5F74696D5F65782E63000061
:101E0000004001400018004010B50446002C58D096
:101E10003648226882422BD0B2F1804F28D0344815
:101E2000824225D03348824222D0334882421FD09A
:101E3000324882421CD03248824219D03148824214
:101E400016D03148824213D03048824210D03048F8
:101E500082420DD02F4882420AD02F48824207D0BA
:101E60002E48824204D04FF489712DA002F084FBE9
:101E7000A06860B110280AD0202808D0402806D0D9
:101E8000602804D040F2131125A002F075FB2069F0
:101E900050B1B0F5807F07D0B0F5007F04D04FF48B
:101EA0008A711FA002F068FBA06930B1802804D0BD
:101EB00040F215111AA002F05FFB94F83D0010B13A
:101EC00007E0012010BD002084F83C00204600F00F
:101ED00043F8022084F83D00211D206801F082FDB6
:101EE000012084F83D00002010BD000000000140EA
:101EF0000004004000080040000C004000100040BA
:101F00000014004000040140004001400044014032
:101F10000048014000180040001C00400020004024
:101F20002E2E2F447269766572732F53544D3332BF
:101F3000463478785F48414C5F4472697665722F09
:101F40005372632F73746D3332663478785F6861CF
:101F50006C5F74696D2E63002DE9F84304464B49AC
:101F60002068002688422DD14948016841F00201CD
:101F70000160006800F002000090474D454828606D
:101F80004FF020606860AE60EE602E614FF48050CC
:101F900068618000A861EE612E626E622846FEF7DD
:101FA000E9FC08B1FEF7EBFB2563AC632562AC638B
:101FB000002211461D20FFF7EBF8BDE8F8431D2075
:101FC000FFF7B2B8354988425ED13148001D01683B
:101FD00041F002010160006800F0020000902E4D07
:101FE0002F48603528604FF06068C5F80480AE6007
:101FF000EE6007152F616E61AE61EE612E626E625A
:102000002846FEF7B7FC08B1FEF7B9FB2563AC63C1
:10201000A563AC636563AC6321481F4D9038C03540
:102020002860C5F80480AE60EE602F614FF4006850
:10203000C5F814804FF40059C5F81890EE612E626F
:102040006E622846FEF796FC08B1FEF798FB256203
:10205000AC631348134D783828606E60AE60EE6054
:102060002F61C5F81480C5F81890EE612E626E627B
:102070002846FEF77FFC08B1FEF781FB6562AC6382
:10208000A562AC63E562AC63BDE8F8830004004080
:102090004038024040600240DC0000200004014063
:1020A000B8640240FC0100202DE9F05F05460C46B3
:1020B00095F83C00012842D0012085F83C00022020
:1020C00085F83D0020684FF40056B0F5805F15D0CC
:1020D000B04213D090B1102810D020280ED0302854
:1020E0000CD040280AD0502808D0602806D070288C
:1020F00004D041F28B11D4A002F03EFA2868816826
:1021000021F0770121F47F418160DE4A2068DC49BB
:10211000DD4BDFF878C3DFF87883DFF87893DFF8FA
:1021200078B3D7134FF0804A50287DD00FDC202899
:1021300004D007DC0028FBD0102852D164E1022033
:10214000BDE8F09F3028F9D04028F6D127E160287B
:102150006BD0702873D0B0F5805F43D0B042ECD123
:10216000286888420ED050450CD090420AD0984240
:1021700008D0604506D0404504D041F2B611B2A067
:1021800002F0FAF9A06860B1B0F5805F09D0B04202
:1021900007D0B0F5405F04D041F2B911AAA002F017
:1021A000EBF96068B84209D040B1022806D00A288D
:1021B00004D041F2BA11A4A002F0DEF9E0680F28C1
:1021C00004D941F2BB11A0A002F0D6F9D4E9021360
:1021D0006268286801F0E6FC2868816841F4804163
:1021E00081602BE128688842FBD05045F9D09042AD
:1021F000F7D09842F5D06045F3D0A8498842F0D096
:10220000A7498842EDD04045EBD04845E9D0A549E3
:102210008842E6D0A4498842E3D05845E1D0A3499A
:102220008842DED0A24902E04FE083E007E0884226
:10223000D7D041F2971184A002F09EF9FEE0286801
:10224000884212D0504510D090420ED098420CD007
:1022500060450AD0404508D0484506D0584504D0CE
:1022600041F29E1178A002F087F9A06860B1B0F544
:10227000805F09D0B04207D0B0F5405F04D041F292
:10228000A11171A002F078F96068B84209D040B19C
:10229000022806D00A2804D041F2A2116AA002F056
:1022A0006BF9E0680F2804D941F2A31166A002F08F
:1022B00063F9D4E902136268286801F073FC2868A6
:1022C000816841F077018160B8E02868884212D0C7
:1022D000504510D090420ED098420CD060450AD0A4
:1022E000404508D0484506D0584504D041F2CA11AF
:1022F00055A002F041F96068B84209D040B1022807
:1023000006D00A2804D041F2CD114FA002F034F9D2
:10231000E0680F2804D941F2CE114BA002F02CF94D
:10232000E2686168286801F00DFE5021286801F01C
:1023300043FC83E02868884212D0504510D0904278
:102340000ED098420CD060450AD0404508D0484590
:1023500006D0584504D041F2DA113BA002F00CF946
:102360006068B84209D040B1022806D00A2804D0DB
:1023700041F2DD1134A002F0FFF8E0680F2804D923
:1023800041F2DE1130A002F0F7F8E26861682868D7
:1023900001F0E9FD6021286801F00EFC4EE028689C
:1023A000884212D0504510D090420ED098420CD0A6
:1023B00060450AD0404508D0484506D0584504D06D
:1023C00041F2EA1120A002F0D7F86068B84209D0C3
:1023D00040B1022806D00A2804D041F2ED111AA01B
:1023E00002F0CAF8E0680F2804D941F2EE1116A0F5
:1023F00002F0C2F8E2686168286801F0A3FD40219C
:10240000286801F0D9FB19E02868884212D05045AD
:1024100010D090420ED098420CD060450AD0404572
:1024200008D0484506D0584504D041F2FD1106A019
:1024300002F0A2F82168286801F0BEFB01203C35BB
:102440006870002028707BE62E2E2F447269766516
:1024500072732F53544D3332463478785F48414C71
:102460005F4472697665722F5372632F73746D3394
:1024700032663478785F68616C5F74696D2E6300D2
:10248000000001400004004000080040000C004033
:1024900000040140004001400018004000100040CE
:1024A000001400400044014000480140001C00406E
:1024B00000200040704770B50446206801694FF065
:1024C0000005C943890716D4C168C943890712D4D6
:1024D000E91E01610120207720688069800703D010
:1024E0002046FFF7E7FF05E0204600F0B9F9204657
:1024F00000F042FC257720680169C943490718D4D8
:10250000C168C943490714D46FF004010161022076
:1025100020772068806910F4407F03D02046FFF7C1
:10252000C9FF05E0204600F09BF9204600F024FC9E
:10253000257720680169C943090717D4C168C943D1
:10254000090713D46FF00801016104202077206887
:10255000C069800703D02046FFF7ACFF05E02046A6
:1025600000F07EF9204600F007FC2577206801691D
:10257000C943C90618D4C168C943C90614D46FF049
:1025800010010161082020772068C06910F4407FA5
:1025900003D02046FFF78EFF05E0204600F060F9EB
:1025A000204600F0E9FB257720680169C943C90787
:1025B00008D1C168C943C90704D1891E01612046F9
:1025C00000F0A0FD20680169C943090609D4C1686B
:1025D000C943090605D46FF0800101612046FFF769
:1025E000C7FA20680169C943490609D4C168C943CB
:1025F000490605D46FF040010161204600F083FDDB
:1026000020680169C94389060BD4C168C94389069A
:1026100007D46FF0200101612046BDE87040FFF74C
:10262000A8BA70BD10B586B00446142101A8FDF704
:1026300011FE0D492068884214D100210B48026820
:1026400042F001020260006800F0010000904020AA
:1026500001900220029003900491059001A9044882
:10266000FEF7F6FA06B010BD000400403038024014
:10267000000002402DE9F05F04460E461546002D8D
:102680000CD0042D0AD0082D08D00C2D06D03C2DDE
:1026900004D040F63B5159A001F06EFF306870B194
:1026A00010280CD020280AD0302808D0502806D076
:1026B000402804D040F63C5150A001F05DFFB068C6
:1026C00030B1022804D040F63D514CA001F054FF37
:1026D00094F83C0001281AD0012784F83C700220AD
:1026E00084F83D005349544A544BDFF854C1DFF895
:1026F0005481DFF854A1DFF854B14FF080494DB157
:10270000042D2ED0082D47D00C2D72D15BE0022075
:10271000BDE8F09F206888421ED048451CD09042FA
:102720001AD0984218D0604516D0404514D0504574
:1027300012D0474988420FD0464988420CD05845AC
:102740000AD04549884207D04449884204D040F61F
:1027500049512AA001F010FF3146206801F034FAF7
:1027600047E02068884212D0484510D090420ED0F1
:1027700098420CD060450AD0404508D0504506D05C
:10278000584504D040F653511CA001F0F5FE3146E7
:10279000206801F08FFA2CE0206888420ED048456E
:1027A0000CD090420AD0984208D0604506D04045EF
:1027B00004D040F65D5111A001F0DEFE31462068E4
:1027C00001F0F2FA15E0206888420ED048450CD09E
:1027D00090420AD0984208D0604506D0404504D0C7
:1027E00040F6675105A001F0C7FE3146206801F0B0
:1027F00055FB3C3467700020207089E72E2E2F4453
:102800007269766572732F53544D3332463478783B
:102810005F48414C5F4472697665722F5372632F33
:1028200073746D3332663478785F68616C5F746995
:102830006D2E6300000001400004004000080040CD
:10284000000C00400004014000400140001800401E
:102850000044014000480140001C004000200040AE
:102860007047000010B50446002C58D03648226846
:1028700082422BD0B2F1804F28D03448824225D0FA
:102880003348824222D0334882421FD032488242AB
:102890001CD03248824219D03148824216D0314889
:1028A000824213D03048824210D0304882420DD04C
:1028B0002F4882420AD02F48824207D02E488242B7
:1028C00004D040F25E212DA001F056FEA06860B158
:1028D00010280AD0202808D0402806D0602804D02C
:1028E00040F25F2125A001F047FE206950B1B0F50C
:1028F000807F07D0B0F5007F04D04FF418711FA07F
:1029000001F03AFEA06930B1802804D040F2612184
:102910001AA001F031FE94F83D0010B107E001204B
:1029200010BD002084F83C00204600F043F802204F
:1029300084F83D00211D206801F054F8012084F83E
:102940003D00002010BD00000000014000040040D8
:1029500000080040000C004000100040001400403F
:102960000004014000400140004401400048014093
:1029700000180040001C0040002000402E2E2F4474
:102980007269766572732F53544D333246347878BA
:102990005F48414C5F4472697665722F5372632FB2
:1029A00073746D3332663478785F68616C5F746914
:1029B0006D2E6300704700002DE9F05F04460D4660
:1029C0001646002E0CD0042E0AD0082E08D00C2E4D
:1029D00006D03C2E04D040F6EC5179A001F0CCFD9D
:1029E0002868602806D0702804D040F6ED5174A005
:1029F00001F0C2FDA86830B1022804D040F6EE51C3
:102A00006FA001F0B9FD286930B1042804D040F668
:102A1000EF516BA001F0B0FD94F83C0001281AD0F2
:102A2000012784F83C70022084F83D007249734A03
:102A3000734BDFF8D0C1DFF8D081DFF8D0A1DFF829
:102A4000D0B14FF080494EB1042E3DD0082E66D053
:102A50000C2E38D189E00220BDE8F09F2068884222
:102A60001ED048451CD090421AD0984218D06045DC
:102A700016D0404514D0504512D0664988420FD038
:102A8000654988420CD058450AD06449884207D02D
:102A90006349884204D040F6FB5149A001F06CFD27
:102AA0002946206801F090F82068816941F008010A
:102AB00081612068816921F0040181612068816958
:102AC0002A691143816176E02068884212D0484526
:102AD00010D090420ED098420CD060450AD04045AC
:102AE00008D0504506D0584504D040F60C6134A0BB
:102AF00001F042FD2946206801F0DCF82068816978
:102B000041F4006181612068816921F48061816103
:102B1000206881692A6941EA022181614BE02068CD
:102B200088420ED048450CD090420AD0984208D036
:102B3000604506D0404504D040F61D6120A001F05C
:102B40001BFD2946206801F02FF92068C16941F07A
:102B50000801C1612068C16921F00401C1612068D8
:102B6000C1692A691143C16125E0206888420ED0FD
:102B700048450CD090420AD0984208D0604506D013
:102B8000404504D040F62E610DA001F0F5FC294629
:102B9000206801F083F92068C16941F40061C161D6
:102BA0002068C16921F48061C1612068C1692A6916
:102BB00041EA0221C1613C346770002020704BE77C
:102BC0002E2E2F447269766572732F53544D333213
:102BD000463478785F48414C5F4472697665722F5D
:102BE0005372632F73746D3332663478785F686123
:102BF0006C5F74696D2E63000000014000040040AA
:102C000000080040000C004000040140004001406A
:102C1000001800400044014000480140001C0040F2
:102C20000020004010B50446002C58D036482268D9
:102C300082422BD0B2F1804F28D03448824225D036
:102C40003348824222D0334882421FD032488242E7
:102C50001CD03248824219D03148824216D03148C5
:102C6000824213D03048824210D0304882420DD088
:102C70002F4882420AD02F48824207D02E488242F3
:102C800004D040F29B412DA001F076FCA06860B119
:102C900010280AD0202808D0402806D0602804D068
:102CA00040F29C4125A001F067FC206950B1B0F5CD
:102CB000807F07D0B0F5007F04D040F29D411FA077
:102CC00001F05AFCA06930B1802804D040F29E4146
:102CD0001AA001F051FC94F83D0010B107E001206A
:102CE00010BD002084F83C00204600F043F802208C
:102CF00084F83D00211D206800F074FE012084F856
:102D00003D00002010BD0000000001400004004014
:102D100000080040000C004000100040001400407B
:102D200000040140004001400044014000480140CF
:102D300000180040001C0040002000402E2E2F44B0
:102D40007269766572732F53544D333246347878F6
:102D50005F48414C5F4472697665722F5372632FEE
:102D600073746D3332663478785F68616C5F746950
:102D70006D2E63007047000000680849884207D143
:102D80000749C878002803D1886810B1401E8860C0
:102D900070470021034800F0D9B80000000400404B
:102DA000000000205C0000202DE9F04105460C46A3
:102DB0004D4E29684D4FB14207D1002C5AD0042CFA
:102DC00058D0082C56D00C2C54D0B1F1804F07D1DC
:102DD000002C4FD0042C4DD0082C4BD00C2C49D0BB
:102DE0004348814206D1ECB3042C43D0082C41D097
:102DF0000C2C3FD03F48814206D19CB3042C39D0E3
:102E0000082C37D00C2C35D03B48814206D14CB32E
:102E1000042C2FD0082C2DD00C2C2BD0B94206D14D
:102E200004B3042C26D0082C24D00C2C22D03348F8
:102E3000814202D1B4B1042C1CD03148814200D16E
:102E400084B13048814200D164B12F48814202D11F
:102E500044B1042C0ED02D48814200D114B12C482D
:102E6000814200E006E000D124B140F25B5129A08C
:102E700001F082FB34B1042C0AD0082C0ED00C2CAB
:102E800017D111E02868C16841F00201C16010E06B
:102E90002868C16841F00401C1600AE02868C1687F
:102EA00041F00801C16004E02868C16841F01001E8
:102EB000C16001222146286800F0FAFD2868B0426E
:102EC00001D0B84203D1416C41F40041416428680B
:102ED000816801F00701062903D0016841F0010172
:102EE00001600020BDE8F0810000014000040140C5
:102EF0000004004000080040000C00400040014079
:102F0000004401400048014000180040001C0040FF
:102F1000002000402E2E2F447269766572732F5365
:102F2000544D3332463478785F48414C5F4472697F
:102F30007665722F5372632F73746D3332663478F3
:102F4000785F68616C5F74696D2E63002DE9F041F4
:102F500005460C46524E2968524FB14207D1002C0B
:102F60005AD0042C58D0082C56D00C2C54D0B1F187
:102F7000804F07D1002C4FD0042C4DD0082C4BD0C3
:102F80000C2C49D04848814206D1ECB3042C43D0E4
:102F9000082C41D00C2C3FD04448814206D19CB330
:102FA000042C39D0082C37D00C2C35D04048814225
:102FB00006D14CB3042C2FD0082C2DD00C2C2BD0A8
:102FC000B94206D104B3042C26D0082C24D00C2CF2
:102FD00022D03848814202D1B4B1042C1CD03648EA
:102FE000814200D184B13548814200D164B1344876
:102FF000814202D144B1042C0ED03248814200D12A
:1030000014B13148814200E006E000D124B140F221
:10301000A1512EA001F0B0FA34B1042C0AD0082C32
:103020000ED00C2C17D111E02868C16821F00201E4
:10303000C16010E02868C16821F00401C1600AE0A5
:103040002868C16821F00801C16004E02868C168EF
:1030500021F01001C16000222146286800F028FDFF
:1030600041F2111128688B10B04201D0B84209D149
:10307000026A0A4206D1026A1A4203D1426C22F461
:10308000004242642868026A0A4206D1016A194273
:1030900003D1016821F0010101600020BDE8F08149
:1030A000000001400004014000040040000800400E
:1030B000000C004000400140004401400048014035
:1030C00000180040001C0040002000402E2E2F441D
:1030D0007269766572732F53544D33324634787863
:1030E0005F48414C5F4472697665722F5372632F5B
:1030F00073746D3332663478785F68616C5F7469BD
:103100006D2E6300704770477047000070B504462D
:1031100022681068D168526900F00F03002B08D1B3
:10312000850606D58D0604D52046BDE8704000F022
:103130004FBF002B61D002F0010301F490751D43D5
:103140005BD0C50705D0CD0503D5E56B45F001057E
:10315000E563450705D5D50703D0E56B45F00205C6
:10316000E563850705D5D20703D0E26B42F0040280
:10317000E263020707D501F020021A4303D0E26B95
:1031800042F00802E263E26B002A2BD0800604D5ED
:10319000880602D5204600F01BFF20684069C0F376
:1031A0008010E16B01F00801014320D0204600F0BF
:1031B000F4FE20684169490615D5416921F04001B6
:1031C0004161606B58B116490165606BFDF7D8FA33
:1031D000002807D0606B016DBDE8704008472046AD
:1031E000FFF792FF70BD2046FFF78EFF70BD2046AF
:1031F000FFF78AFF0020E06370BD020606D50A06CD
:1032000004D52046BDE8704001F06AB84006F3D509
:103210004806F1D52046BDE8704000F0CCBE000065
:103220008B3F000870B50446002C26D0A0694049A9
:10323000404A414B414D002821D0206888420AD0A5
:10324000904208D0984206D0A84204D040F24B11D8
:103250003BA001F091F9A06900282AD0B0F5807F49
:1032600027D0B0F5007F24D0B0F5407F21D04FF4B7
:10327000A67133A001F080F91BE0012070BD206829
:10328000884216D0904214D0984212D03B498842CE
:103290000FD03B4988420CD0A8420AD03949884215
:1032A00007D03949884204D04FF4A87124A001F016
:1032B00063F9A06838B1B0F5805F04D04FF4A9710C
:1032C0001FA001F059F9E06938B1B0F5004F04D002
:1032D00040F253111AA001F04FF994F8390000257B
:1032E00020B984F83850204600F050F8242084F8A3
:1032F00039002068C16821F40051C160204600F007
:10330000B5FE2068016921F490410161206841699E
:1033100021F02A0141612068C16841F40051C16077
:10332000E563202084F8390084F83A00002070BD5D
:1033300000100140004400400048004000140140DB
:103340002E2E2F447269766572732F53544D33328B
:10335000463478785F48414C5F4472697665722FD5
:103360005372632F73746D3332663478785F68619B
:103370006C5F756172742E6300000000004C0040A9
:103380000050004000780040007C0040F0B587B05D
:103390000446142102A8FCF75DFF274F2168002690
:1033A000264A0223032407252548B94224D123496C
:1033B00014310F6847F010070F60096801F0100121
:1033C0000191116841F001011160116801F00101E2
:1033D000019161020291039304960594069502A956
:1033E000FDF736FC002211462520FDF7D1FE2520F1
:1033F000FDF79AFE07B0F0BD124FB942FAD10F495E
:1034000010310F6847F400370F60096801F400318C
:103410000191116841F001011160116801F0010191
:1034200001910C210291039304960594069502A93B
:10343000FDF70EFCDEE700000010014030380240CE
:10344000000002400044004090F83A30202B01D0A8
:1034500002207047F9B1F2B190F83830012B1CD03E
:1034600081628285C2850021C163222280F83A20D0
:1034700080F838100168CA6842F48072CA60016836
:103480004A6942F001024A610068C16841F02001C6
:10349000C160002070470120704702207047000083
:1034A00010B50D49814213D10C4B987800280FD1EB
:1034B0001846197840780A4C421CD2B2532908D0D9
:1034C00008B121545A705878142801D101209870FD
:1034D00010BD21545A70F6E75C0200200000002065
:1034E000280000202DE9F84304460D4690461E466C
:1034F00094F83900202802D00220BDE8F883D5B125
:10350000B8F1000F17D094F83800012815D0012029
:1035100084F838004FF00009C4F83C90212084F86A
:103520003900FDF79FFD0746A4F82480A4F8268003
:1035300084F838902DE00120DFE70220DDE7E08C01
:10354000401EE084A068B0F5805F09D03B460022B1
:1035500080212046009600F0F6FEB0B10320CCE7B3
:103560003B46002280212046009600F0ECFE08B188
:103570000320C2E728882168C0F30800486020695A
:1035800008B16D1C05E0AD1C03E0216815F8010BC6
:103590004860E08C0028D2D13B46002240212046E2
:1035A000009600F0D0FE08B10320A6E7202084F8A2
:1035B00039000020A1E77047FEE7000008B5194870
:1035C000016841F480010160016801F4800100910B
:1035D000016841F400110160006800F400100090DF
:1035E000002211460D20FDF7D3FD0D20FDF79CFDB7
:1035F000002211463920FDF7CBFD3920FDF794FD5F
:10360000002211463A20FDF7C3FD3A20FDF78CFD5C
:10361000002211464620FDF7BBFDBDE808404620CC
:10362000FDF782BD303802402DE9F04387B0142108
:1036300002A8FCF70FFE00243E48016841F010018B
:103640000160016801F010010191016841F004017D
:103650000160016801F004010191016841F08001FD
:103660000160016801F080010191016841F00101F0
:103670000160016801F001010191016841F002015E
:103680000160016801F002010191016841F0080147
:103690000160006800F008000190DFF89C800022C3
:1036A00003214046FDF7A6FCDFF89090002202219E
:1036B0004846FDF79FFC4FF6FF76029603250395DB
:1036C000049402A91E48FDF7C3FAF01E0290039568
:1036D000049402A94046FDF7BBFA0295012703971F
:1036E0000494059402A94046FDF7B2FA49F6B110D8
:1036F00002900395049402A94846FDF7A9FA022016
:10370000029003970494059402A94846FDF7A0FA95
:1037100002960395049402A90A48FDF799FA0296C5
:103720000395049402A90848FDF792FA07B0BDE892
:10373000F0830000303802400008024000000240E0
:103740000010024000040240000C024010B58EB090
:1037500000240A940B940C940D94089409941C2151
:1037600001A8FCF777FD1D481B4901604460846097
:103770000121C16004618461FEF746FB08B1FCF7DA
:10378000FEFF4FF480500A900AA91448FEF78CFC03
:1037900008B1FCF7F4FF1148FFF744FA08B1FCF751
:1037A000EEFF0894099408A90C48FEF787FA08B1BF
:1037B000FCF7E5FF60200190029403940594002239
:1037C00001A90648FFF7F8F808B1FCF7D8FF03484D
:1037D000FEF728FF0EB010BD000400405C00002082
:1037E00010B596B000241294139414941594109468
:1037F00011941C2109A8FCF72DFD202101A8FCF73C
:1038000029FD25482349016044608460C460046147
:1038100044618461FEF7F8FA08B1FCF7B0FF4FF499
:103820008050129012A91C48FEF73EFC08B1FCF72C
:10383000A6FF1948FFF716F808B1FCF7A0FF10948F
:10384000119410A91448FEF739FA08B1FCF797FF54
:1038500009940A940B940C940D940E940F940022E6
:1038600009A90D48FEF706FF08B1FCF788FF01948F
:1038700002940394049405944FF400500690089425
:1038800001A90548FEF776F9002801D0FCF777FF7B
:1038900016B010BD000401409C00002010B50C487B
:1038A0000A4901604FF41651416000218160C160F6
:1038B00001610C2242618161C161FFF7B3FC002804
:1038C00003D0BDE81040FCF75ABF10BD0010014006
:1038D0005C02002010B50C480A4901604FF41651F3
:1038E000416000218160C16001610C2242618161FF
:1038F000C161FFF797FC002803D0BDE81040FCF73A
:103900003EBF10BD004400409C020020FEE770470F
:1039100070477047FDF7ACBB30B593B0302107A8B6
:10392000FCF798FC142102A8FCF794FC0025214820
:10393000016841F080510160006800F08050019002
:103940001D48016841F440410160006800F44040B6
:1039500001900A20079001200A9010210B910C90F1
:1039600002240D940E9508200F90B420109011940D
:103970000420129007A8FDF769FE08B1FCF7FFFECE
:10398000FDF796FC08B1FCF7FAFE0F2002900394B5
:1039900004954FF4A05005904FF4805006900521F7
:1039A00002A8FDF7BFFC002801D0FCF7E8FE13B029
:1039B00030BD0000403802400070004005480168FA
:1039C00041F47001016003494FF0006080390860E4
:1039D0007047000088ED00E00148FEF76CBD000074
:1039E0005C0000202DE9F0410268264D264E274F4D
:1039F000DFF89CC0274B4FF08048A84209D04045D3
:103A000007D0B04205D0B84203D0604501D09842FB
:103A100003D122F070044A682243A8421BD04045DB
:103A200019D0B04217D0B84215D0604513D0984293
:103A300011D0194CA0420ED0184CA0420BD0184CFB
:103A4000A04208D0174CA04205D0174CA04202D08B
:103A5000164CA04203D122F44074CA6822434C6938
:103A600022F08002224302608A68C2620A6882628F
:103A7000A84201D0984201D1096901630121416145
:103A8000BDE8F08100000140000400400008004053
:103A9000000C00400004014000400140004401408F
:103AA0000048014000180040001C00400020004079
:103AB00070B504460D4616462148844225D0B4F11F
:103AC000804F22D01F4884421FD01F4884421CD000
:103AD0001E48844219D01E48844216D01D48844294
:103AE00013D01D48844210D01C4884420DD01C487D
:103AF00084420AD01B48844207D01B48844204D029
:103B000041F6CC1119A000F037FD65B1042D0AD0A3
:103B1000082D08D00C2D06D03C2D04D041F6CD1137
:103B200012A000F029FD05F01F0001218140226A4A
:103B30008A432262216A86403143216270BD0000BF
:103B4000000001400004004000080040000C00405C
:103B50000004014000400140004401400048014091
:103B600000180040001C0040002000402E2E2F4472
:103B70007269766572732F53544D333246347878B8
:103B80005F48414C5F4472697665722F5372632FB0
:103B900073746D3332663478785F68616C5F746912
:103BA0006D2E630010B5846824F47F4442EA03223A
:103BB0000A432243826010BD826822F070020A43E9
:103BC00042F00701816070472DE9F04704460D4639
:103BD000206A20F001002062206A6768A16921F054
:103BE000700121F00301D5F8008048EA010820F0B7
:103BF0000200AE680643DFF87C90DFF87CA04C45FD
:103C000001D054450ED1E86830B1082804D041F203
:103C100002711AA000F0B0FC26F00801E868084321
:103C200020F004064C4501D054451BD1A869B0F5DD
:103C3000007F05D020B141F20F7110A000F09CFC74
:103C40006869B0F5807F05D020B141F210710BA0FA
:103C500000F092FC27F4807020F40071686908433A
:103C6000AF6907436760C4F81880686860632662BC
:103C7000BDE8F08700000140000401402E2E2F44D3
:103C80007269766572732F53544D333246347878A7
:103C90005F48414C5F4472697665722F5372632F9F
:103CA00073746D3332663478785F68616C5F746901
:103CB0006D2E63002DE9F04704460D46206A20F082
:103CC00010002062206A6768A16921F4E04121F4B4
:103CD00040712A6841EA022820F02000A96840EAE1
:103CE0000116DFF88490DFF884A04C4501D05445DC
:103CF0000FD1E86830B1082804D041F24D711CA002
:103D000000F03AFC26F08000E96840EA011020F05B
:103D100040064C4501D054451DD1A869B0F5007F3F
:103D200005D020B141F25B7111A000F025FC68695B
:103D3000B0F5807F05D020B141F25C710CA000F09D
:103D40001BFC27F4806020F40060696940EA810070
:103D5000A96940EA81076760C4F818806868A063B1
:103D60002662BDE8F0870000000001400004014029
:103D70002E2E2F447269766572732F53544D333251
:103D8000463478785F48414C5F4472697665722F9B
:103D90005372632F73746D3332663478785F686161
:103DA0006C5F74696D2E63002DE9F04704460D4683
:103DB000206A20F480702062206A6768E16921F03F
:103DC000700121F00301D5F8008048EA010820F4D1
:103DD0000070A96840EA0126DFF88090DFF880A033
:103DE0004C4501D054450FD1E86830B1082804D0C3
:103DF00041F298711BA000F0BFFB26F40060E96857
:103E000040EA012020F480664C4501D054451DD184
:103E1000A869B0F5007F05D020B141F2A57111A0CD
:103E200000F0AAFB6869B0F5807F05D020B141F2AF
:103E3000A6710CA000F0A0FB27F4805020F40050E5
:103E4000696940EA0110A96940EA01176760C4F88E
:103E50001C806868E0632662BDE8F08700000140CE
:103E6000000401402E2E2F447269766572732F5321
:103E7000544D3332463478785F48414C5F44726920
:103E80007665722F5372632F73746D333266347894
:103E9000785F68616C5F74696D2E63002DE9F04195
:103EA00004460D46206A20F480502062206A66682D
:103EB000E16921F4E04121F440712A6841EA0227D6
:103EC00020F40050A96840EA01380E48844202D02C
:103ED0000D4884420ED16869B0F5807F05D020B1CD
:103EE00041F2E47109A000F047FB26F480406969C3
:103EF00040EA81166660E76168682064C4F8208043
:103F0000BDE8F08100000140000401402E2E2F4446
:103F10007269766572732F53544D33324634787814
:103F20005F48414C5F4472697665722F5372632F0C
:103F300073746D3332663478785F68616C5F74696E
:103F40006D2E630010B5036A046A24F00104046254
:103F5000846924F0F00444EA021423F00A020A43BC
:103F60008461026210BD10B5036A23F0100303627E
:103F70008469036A24F4704444EA023223F0A00303
:103F800043EA01118261016210BD10B5806B00210E
:103F9000C185C184FFF7B8F810BD0168CA6822F472
:103FA0009072CA6001684A6922F001024A612021C8
:103FB00080F83A10704710B50168CA6822F04002D4
:103FC000CA60202180F83910FFF7F5FA002010BDF3
:103FD00010B590F83A10222901D0022010BD816856
:103FE000B1F5805F11D0016919B30168496801F02A
:103FF0007F03816A4A1C82620B70C18D491E0904CD
:10400000090CC1851CD0002010BD816A02693AB13B
:1040100002685268D2B20A80816A491C8162ECE768
:1040200002685268C2F308020A80816A891C8162B0
:10403000E3E701684A68816A4B1C83620A70DCE727
:104040000168CA6822F02002CA600168CA6822F4C6
:104050008072CA6001684A6922F001024A61202127
:1040600080F83A10FFF71CFA002010BD2DE9F0414E
:10407000044689496068884204D940F6FB3187A02C
:1040800000F07AFAE06838B1B0F5005F04D040F68D
:10409000FC3182A000F070FA206950B1B0F5806F59
:1040A00007D0B0F5C06F04D040F6FD317BA000F022
:1040B00063FA60694FF6F371084200D120B940F607
:1040C000FE3176A000F058FA20680169E26821F418
:1040D000405111430161A1682069E26901436069AF
:1040E000104301432068C26849F20C639A430A43B3
:1040F000C26020684169A26921F4407111434161A5
:10410000E069754A75491927642532264FF0000881
:10411000B0F5004F32D02068884201D090427CD167
:10412000FDF74EFA01466068830F8200A1FB07018C
:10413000FCF758F80146B0FBF5F06FF01802504359
:1041400001EB800006EB0010B0FBF5F000F0F00290
:10415000B1FBF5F002EB0012B1FBF5F06FF01803C4
:10416000584301EB800006EB0010B0FBF5F021682E
:1041700000F00F0010448860BDE8F081206888429C
:1041800001D090422CD1FDF71BFA0146606802185D
:10419000A1FB070148EB0803FCF724F80146B0FB3C
:1041A000F5F00201B1FBF5F06FF01803584301EB95
:1041B000800006EBC000B0FBF5F000F0F80002EB69
:1041C0004002B1FBF5F0584301EB800006EBC00064
:1041D000B0FBF5F0216800F0070010448860CBE7E1
:1041E000FDF7DEF9014660680218A1FB070148EB04
:1041F0000803FBF7F7FF0146B0FBF5F00201B1FB46
:10420000F5F06FF01803584301EB800006EBC00097
:10421000B0FBF5F000F0F80000E010E002EB400227
:10422000B1FBF5F0584301EB800006EBC000B0FB9A
:10423000F5F0216800F00700104488609CE7FDF766
:10424000AFF901466068830F8200A1FB0701FBF70D
:10425000C9FF0146B0FBF5F06FF01802504301EBC7
:10426000800006EB0010B0FBF5F000F0F002B1FBAF
:10427000F5F002EB0012B1FBF5F06FF018035843B4
:1042800001EB800006EB0010B0FBF5F0216800F0B8
:104290000F00104488606FE7A037A0002E2E2F4437
:1042A0007269766572732F53544D33324634787881
:1042B0005F48414C5F4472697665722F5372632F79
:1042C00073746D3332663478785F68616C5F7561E2
:1042D00072742E63000000000014014000100140C1
:1042E00090F83910212901D0022070478168B1F57A
:1042F000805F0CD0016A4A1C026202680978516032
:10430000C18C491E0904090CC18410D019E0016A4E
:1043100002680988C1F308015160016919B1016A95
:10432000491C0162ECE7016A891C0162E8E7016847
:10433000CA6822F08002CA600068C16841F040018A
:10434000C160002070472DE9F04104460E46174633
:104350009846069D1DE0681C1BD02DB1FCF782FE1F
:10436000A0EB0800A84214D92068C16821F4D071DC
:10437000C1602068416921F001014161202084F879
:10438000390084F83A00002084F838000320BDE8A2
:10439000F0812068006836EA000004D00020B842AE
:1043A000D9D00020F3E70120F9E700000148FEF72B
:1043B000ADBE00005C020020FEE700000FB4054B1C
:1043C00010B503A9044A029800F02CF810BC5DF85F
:1043D00014FB00007D450008200000200907090E9D
:1043E000002804DB00F1E02080F80014704700F0A2
:1043F0000F0000F1E02080F8141D7047004870475E
:104400002400002002E008C8121F08C1002AFAD1C7
:1044100070477047002001E001C1121F002AFBD144
:10442000704700002DE9FF4F89B09B4604460025E8
:1044300006E025280BD05A460B999047641C6D1C4A
:1044400020780028F5D10DB02846BDE8F08F002770
:10445000B8460122474900E0074314F8013F203BDA
:1044600002FA03F00842F7D120782E2819D114F867
:10447000010F47F004072A280ED06FF02F02207892
:10448000A0F1300109290CD808EB880102EB4101A9
:1044900000EB0108641CF2E70A98641C50F8048BD6
:1044A0000A9020780028CED0642808D0692806D049
:1044B00075281ED05A460B9990476D1C58E00A99F2
:1044C0004FF00A0901C90A91002802DA40422D2161
:1044D00002E0390504D52B218DF82010012103E0DD
:1044E000F90704D02021F7E78A4608AE0DE0002145
:1044F000FAE70A994FF00A0901C90A91F7E7494614
:10450000FBF75CFF303106F8011D0028F7D1ADEB59
:10451000060000F12009780701D44FF00108C845D2
:1045200002DDA8EB090000E000208046002706E03D
:1045300008A85A46C05D0B9990476D1C7F1C5745D3
:10454000F6DB04E030205A460B9990476D1CB8F119
:104550000001A8F10108F5DC05E016F8010B5A4648
:104560000B9990476D1CB9F10001A9F10109F4DC28
:10457000641C65E7092801007047000038B504464F
:1045800000946423012269460248FEF7ABFF2046EF
:1045900038BD00005C020020FCF772FDFFF7BCF99B
:1045A000FFF742F8FFF70AF8FFF7D0F8FFF718F91E
:1045B000FFF774F9FFF78EF900F01CF9FEE710B56C
:1045C0000446FCF74FFDA04201D3001B10BDE143A0
:1045D000084410BD70B52DED028B86B0002005900B
:1045E000039001902C480168049101798DF8141012
:1045F000D0F805100291B0F80910ADF80C10C17A8E
:104600008DF80E10C1680091018AADF80410807C0D
:104610008DF8060004A8FBF728FE044602A8FBF765
:1046200024FE05466846FBF720FE064600F05EF8CD
:104630002046FBF796FE41EC100B53EC102B9FED40
:10464000170B51EC100BFBF71DFE41EC180B284625
:10465000FBF787FE9FED131B53EC112BFBF712FEAC
:1046600053EC182BFBF70EFEFBF78CFE08EE100A3E
:1046700021460EA0FFF7A2FE0A2095FBF0F10EA046
:10468000FFF79CFE3146B0EE480A204600F042F8A3
:1046900006B0BDEC028B70BD2900002000000000B8
:1046A00080842E410000000000002440665B2564E9
:1046B0005D687A200D0A0000775B25645D757320C4
:1046C0000D0A000010B5074C002201212046FCF71E
:1046D00091FC012202212046FCF78CFC02490020BB
:1046E000087110BD000802400000002010B5074C02
:1046F000012211462046FCF77DFC002202212046C3
:10470000FCF778FC02490120087110BD0008024046
:104710000000002070B504462DED028BB0EE408AFB
:104720000D4600213048FEF711FC002C59D02F48CF
:1047300090FBF4F000EE100AF8EEC00A4FF6FE709F
:10474000044601EE100AB8EE411AC0EE811ABCEE22
:10475000E11A11EE102A5AB101EE102AB8EE411AF0
:10476000C0EE811ABCEEE11A11EE103AA34202D358
:10477000401E0228E5D8002A33D0032831D901EEA3
:10478000102AB8EE410A80EE801AFCEEC10A10EE43
:10479000900A401E521E14490B68D862C8600B680C
:1047A0009A6200EE900AB8EE600A28EE000ABCEEAB
:1047B000C00A10EE100A80B20A6850630C4800224A
:1047C00065B16D1E8560C270086842620021BDEC53
:1047D000028B0548BDE87040FEF7E6BA0123C370BE
:1047E000F2E7BDEC028B70BD5C000020804A5D05E5
:1047F00000000020012214491448FEF725FEFFF7AF
:1048000061FF124E104CDFF8488000254FF4967778
:10481000A07818B1FFF7DEFEA570657096F83A0033
:10482000202804D1012208490848FEF70DFEE0685F
:10483000FFF7C5FEB842EBD9FCF714FCE06002219B
:104840004046FCF7A5FBE3E7000000205C020020E7
:1048500000000240000610160006101600000000BE
:104860000000000001020304060708090000000020
:10487000010203040040404040404040404041416C
:104880004141414040404040404040404040404025
:1048900040404040400502020202020202020202BF
:1048A00002020202022020202020202020202002BC
:1048B000020202020202909090909090101010104C
:1048C00010101010101010101010101010101010E8
:1048D000020202020202888888888888080808087C
:1048E0000808080808080808080808080808080848
:1048F0000202020240000000754800081C4900083E
:10490000000000202800000004440008444900087A
:1049100028000020B8120000144400080000000025
:104920000000000000000000000000000100000086
:1049300010000000000000000024F400000000004F
:044940000000000073
:04000005080001AD41
:00000001FF
